:020000020000FC
:100000000C942B000C942A000C942A000C942A00C7
:100010000C942A000C942A000C942A000C942A00B8
:100020000C942A000C942A000C942A000C942A00A8
:100030000C942A000C942A000C942A000C942A0098
:100040000C942A000C942A000C942A000C942A0088
:100050000C942A0018956FE578E06DBF7EBF789408
:1000600062E061BB02E0102F109562B3602B62BBAF
:1000700062B3612362BB0E94560062B3602B62BB15
:100080000E94560062B3612362BB0E94560062B3B5
:10009000602B62BB0E9456000E9456000E945600D0
:1000A0000E9456000E9456000C9438008EE170E0C9
:1000B00060E06A95F1F77A95D9F78A95C1F70895C6
:00000001FF
